:1000000012C018951895189589C0189518951895C7
:100010001895189518951895189518951895189578
:100020001895189518958FE58DBFC0E4E8E34E2E1E
:1000300084E08EBFD4E0F4E05F2EEEEFF3E0A0E6C4
:10004000B0E088278D933197E9F730D2662480E0BD
:1000500087BB87E088BB85E085BD88E082BD85E001
:1000600086B9EAE7F0E088E469D258E0C895802DC7
:100070005FD231965A95D1F704C00C12120C202091
:100080002020EAE9F0E080E559D258E0C895802DBB
:100090004FD231965A95D1F704C0070F1C18181883
:1000A0001818EAEBF0E088E649D258E0C895802DB0
:1000B0003FD231965A95D1F704C018181818181C59
:1000C0000F07EAEDF0E080E639D258E0C895802DC0
:1000D0002FD231965A95D1F704C020202020030753
:1000E0001E1CEAEFF0E088E529D258E0C895802D83
:1000F0001FD231965A95D1F704C01C1E0703202049
:100100002020379A789489B7806489BF85E085BDBF
:10011000B9D18CE013D2FFCFF894FFCF0F921F928A
:100120002F923F924F925F927F92AF92BF920F9326
:100130001F932F933F934F935F936F937F938F936F
:100140009F93AF93BF93CF93DF93EF93FF938FB7BB
:100150008F9380E087B92DD2A3E6B0E08D939C9376
:10016000A3E6B0E00D911C9142E050E063D1A3E61C
:10017000B0E04D935C9381E087B91BD2A5E6B0E077
:100180008D939C93A5E6B0E00D911C9142E050E068
:1001900051D1A5E6B0E04D935C93A7E6B0E08C9119
:1001A0008F5F8C9300916700023010F009F001C05E
:1001B00003C081E080936700A0E6B0E08C918F5F80
:1001C0008C93009160000B3310F009F001C02AC03D
:1001D000A1E6B0E08C918F5F8C9380E0809360000B
:1001E000009161000B3310F009F001C01BC0A2E6C2
:1001F000B0E08C918F5F8C9380E08093610080E011
:100200008093600000916200073110F009F001C096
:1002100009C080E08093620080E08093600080E00D
:10022000809361000027A6E3B0E08C9182FB0EF47E
:1002300001E040E0041709F004C080E08093600012
:1002400046C00027A6E3B0E08C9180FB0EF401E0ED
:1002500040E0041709F021C0A1E6B0E08C918F5F67
:100260008C93A8E6B0E08C918F5F8C93009168002E
:10027000053010F009F001C005C0A1E6B0E08C9196
:100280008E5F8C93009161000B3310F009F001C078
:1002900003C080E0809361001AC00027A6E3B0E0AD
:1002A0008C9181FB0EF401E040E0041709F00FC0CF
:1002B000A2E6B0E08C918F5F8C93009162000731D1
:1002C00010F009F001C003C080E0809362000027B5
:1002D000A6E3B0E08C9180FB0EF401E041E004174E
:1002E00009F003C081E0809368008FE711E0D9D066
:1002F000EAE9F6E0C1D0009162000A3008F00AC0D5
:10030000ECE9F6E0B9D0A0E2B4E0E2E6F0E07BD1BF
:10031000ABD006C0A0E2B4E0E2E6F0E074D1A4D035
:1003200000916700013009F004C0EEE9F6E0A4D0C6
:1003300003C0E0EAF6E0A0D0009161000A3008F0C6
:100340000AC0ECE9F6E098D0A0E2B4E0E1E6F0E023
:100350005AD18AD006C0A0E2B4E0E1E6F0E053D181
:1003600083D0E2EAF6E088D0E4EAF6E085D0A0E2C5
:10037000B4E0E5E6F0E038D177D08FEB11E091D032
:10038000EAEAF6E079D0A0E2B4E0E3E6F0E02CD1CE
:100390006BD08FEB1EE085D081E0CAD085E0C8D05D
:1003A00084E0C6D08FE71EE07CD081E0C1D082E03F
:1003B000BFD083E0BDD08F918FBFFF91EF91DF91D0
:1003C000CF91BF91AF919F918F917F916F915F91ED
:1003D0004F913F912F911F910F91BF90AF907F90C0
:1003E0005F904F903F902F901F900F90189500FCBA
:1003F00010D0089503D01ED001F8F9CF0024E8945E
:1004000057FF02C009D0689400F80BD010F80124FF
:10041000089502D009D00895509540954F5F5F4FE1
:100420000895E89417FF0895009510950F5F1F4FEA
:1004300068940895352F242FE894452B11F468947F
:100440000895512F402F0027112780E1440F551F99
:10045000001F111F021B130B416018F4020F131F22
:100460004E7F8A9599F70895A0E2B4E08D91882394
:1004700011F05ED0FBCF0895A5D0802D11F058D09B
:10048000FBCF089581E05AD00ED080E857C08FE7A7
:10049000213039F08FEB223021F08FE8233009F042
:1004A0008FEC810F4BC083E0992774C08AEF90E0F6
:1004B00071D08F9A8E9A8D9A8C9A8A9A8B9A9398E9
:1004C00085E090E067D0929897989698959A949A3C
:1004D000929AEF93FF93E0E6F0E050D0FF91EF9116
:1004E000929855D0929AEF93FF93E0E6F0E046D0D1
:1004F000FF91EF9192984BD0929AEF93FF93E0E6A1
:10050000F0E03CD0FF91EF91929841D09498929A6C
:10051000EF93FF93E0E6F0E031D0FF91EF919298F6
:1005200036D088E20BD08EE009D086E007D008955F
:10053000939A829505D004D02AD008959398F9CF44
:10054000859510F4949A01C09498859510F4959A25
:1005500001C09598859510F4969A01C09698859556
:1005600010F4979A01C09798929AEF93FF93E0E660
:10057000F0E004D0FF91EF91929808953197F1F750
:100580000895689462F80895E89462F8089581E007
:1005900090E000C0EF93FF93EE27E82BE92B31F0BA
:1005A000E8EEF3E03197F1F70197D1F7FF91EF9182
:1005B0000895369A3699FECF369A3699FECF84B191
:1005C00095B10895C895319600200895000F111F28
:1005D000221F331F089500951095209530950F5FC9
:1005E0001F4F2F4F3F4F0895019110810EC0019171
:1005F0001191219130810BC00191108117FF05C02D
:100600003FEF2FEF04C0008111272227332737FF48
:1006100003C0E1DF8DE28D93CF93DF93CF92DF9222
:10062000EF92AA24BB24CC24DD24EE2440E2CAE0CD
:10063000DD2755E093E38881890F87FD9F7083FD57
:10064000907F891B89935A95A9F7C0DFAA1CBB1C10
:10065000CC1CDD1CEE1C4A9551F7E894EFE0FF2717
:1006600082910ED0EB30E0F71EF068948A2D0CD00A
:1006700088278D93EF90DF90CF90DF91CF910895F1
:10068000982F829501D0892F8F70805D26F080335E
:1006900009F4089568948D9308953C00300020007B
:1006A0003A003E005475723A000054656D702E5247
:0606B000657475723A004A
:00000001FF
